:020000040000FA
:040800005DEF06F0B2
:1008100003B207EF05F0F2B422EF05F09EB02AEF25
:1008200005F09EB232EF05F0F2A81AEF04F0F2B232
:100830001CEF04F03BEF06F0CD90F2929EA026EF65
:1008400004F00101463F26EF04F0472B9DC1A1F1C2
:100850009EC1A2F19FC1A3F1A0C1A4F199C19DF1D4
:100860009AC19EF19BC19FF19CC1A0F195C199F1E4
:1008700096C19AF197C19BF198C19CF191C195F1F4
:1008800092C196F193C197F194C198F18DC191F104
:100890008EC192F18FC193F190C194F189C18DF114
:1008A0008AC18EF18BC18FF18CC190F185C189F124
:1008B00086C18AF187C18BF188C18CF1CECF85F1D9
:1008C000CFCF86F146C187F147C188F1CF6ACE6AA2
:1008D0000101466B476B9E90CD800EBC0E8E0EBA0A
:1008E00075EF04F00E8A3BEF06F00E8C0EBEB1EFF2
:1008F00004F085C189F186C18AF187C18BF188C175
:100900008CF189C18DF18AC18EF18BC18FF18CC1BF
:1009100090F18DC191F18EC192F18FC193F190C18F
:1009200094F191C195F192C196F193C197F194C15F
:1009300098F195C199F196C19AF197C19BF198C12F
:100940009CF199C19DF19AC19EF19BC19FF19CC1FF
:10095000A0F19DC1A1F19EC1A2F19FC1A3F1A0C1CF
:10096000A4F10101516B526B536B546B85515127AC
:10097000865152238751532388515423895151273B
:100980008A5152238B5153238C5154238D5151271B
:100990008E5152238F5153239051542391515127FB
:1009A00092515223935153239451542395515127DB
:1009B00096515223975153239851542399515127BB
:1009C0009A5152239B5153239C5154239D5151279B
:1009D0009E5152239F515323A0515423A15151277B
:1009E000A2515223A3515323A4515423D8905433DA
:1009F000533352335133D8905433533352335133EA
:100A0000D89054335333523351333BEF06F00392B3
:100A1000030103EE00F080517F0BE92604C0EFFFD5
:100A2000802B8151805D700BD8A48B820000805197
:100A3000815D700BD8A48B9281518019D8B4079036
:100A40003BEF06F0F2940101383F3BEF06F0392B03
:100A50003BEF06F09E900101463F3BEF06F0472B2F
:100A60003BEF06F09E92C3CF48F1C4CF49F1C2825A
:100A700007B49DEF05F03AC13EF13BC13FF13CC1E7
:100A800040F13DC141F151C155F152C156F153C13F
:100A900057F154C158F185C1A5F186C1A6F187C1AE
:100AA000A7F188C1A8F189C1A9F18AC1AAF18BC1B6
:100AB000ABF18CC1ACF18DC1ADF18EC1AEF18FC186
:100AC000AFF190C1B0F191C1B1F192C1B2F193C156
:100AD000B3F194C1B4F195C1B5F196C1B6F197C126
:100AE000B7F198C1B8F199C1B9F19AC1BAF19BC1F6
:100AF000BBF19CC1BCF19DC1BDF19EC1BEF19FC1C6
:100B0000BFF1A0C1C0F1A1C1C1F1A2C1C2F1A3C195
:100B1000C3F1A4C1C4F1010148514E2749514F23EB
:100B2000E86A50230D2E9DEF05F04FC14AF150C1E8
:100B30004BF14E6B4F6B506B078E0201002F3BEF5A
:100B400006F03C0E006F01017967AEEF05F07A67A1
:100B5000AEEF05F07B67AEEF05F07C67B2EF05F016
:100B6000E2EF05F07DC100F17EC101F17FC102F12C
:100B700080C103F10101010E046F000E056F000E2C
:100B8000066F000E076FB0EC13F000C17DF101C1DC
:100B90007EF102C17FF103C180F10067D7EF05F05C
:100BA0000167D7EF05F00267D7EF05F00367E2EFC3
:100BB00005F079C17DF17AC17EF17BC17FF17CC105
:100BC00080F10E80D57ED5BE54D0D6CF3AF1D7CFA6
:100BD0003BF138C13CF1E86AE8CF3DF10F800101FB
:100BE00047A7FFEF05F00E9A0E9C0E9E0101000E26
:100BF000516F600E526F3D0E536F080E546F01011E
:100C00003ABF0FEF06F03B670FEF06F03C670FEFC0
:100C100006F03D670FEF06F0F28834EF06F0F29829
:100C2000516B526B536B546B856B866B876B886B08
:100C3000896B8A6B8B6B8C6B8D6B8E6B8F6B906BF8
:100C4000916B926B936B946B956B966B976B986BA8
:100C5000996B9A6B9B6B9C6B9D6B9E6B9F6BA06B58
:100C6000A16BA26BA36BA46BD76AD66A0101386B28
:100C7000396B3BEF06F002C0E0FF005001C0D8FF27
:100C80001000A6B241EF06F00CC0A9FF0BC0A8FFF0
:100C9000A69EA69CA684F29E550EA76EAA0EA76ECF
:100CA000A682F28EA694A6B253EF06F01200A96EA9
:100CB000A69EA69CA680A8501200076A0E6A0F6A1C
:100CC0000F010E0EC16E860EC06E030EC26E0F01B6
:100CD000896A110E926E080E8A6EF10E936E8B6AFF
:100CE000800E946EF18E0D6A01014E6B4F6B506B4E
:100CF0004A6B4B6BF29A01013A6B3B6B3C6B3D6B61
:100D00003E6B3F6B406B416B426B436B446B456B7F
:100D1000386B396BD76AD66A0F01280ED56EF28A06
:100D2000B00ECD6E9D800101516B526B536B546BB5
:100D3000556B566B576B586B596B5A6B5B6B5C6B97
:100D40000E9A0E9C0E9E760ECA6E9D8202013C0E7D
:100D5000006FCC6A160E57EC06F0E8CF00F1170EC4
:100D600057EC06F0E8CF01F1180E57EC06F0E8CF8B
:100D700002F1190E57EC06F0E8CF03F1010103AFC1
:100D8000DCEF06F0A7EC14F0160E0C6E00C10BF0B1
:100D900041EC06F0170E0C6E01C10BF041EC06F0B1
:100DA000180E0C6E02C10BF041EC06F0190E0C6E21
:100DB00003C10BF041EC06F000C179F101C17AF1F9
:100DC00002C17BF103C17CF100C17DF101C17EF163
:100DD00002C17FF103C180F11A0E57EC06F0E8CF93
:100DE00000F11B0E57EC06F0E8CF01F11C0E57EC9A
:100DF00006F0E8CF02F11D0E57EC06F0E8CF03F144
:100E0000010103AF32EF07F0A7EC14F01A0E0C6EDD
:100E100000C10BF041EC06F01B0E0C6E01C10BF093
:100E200041EC06F01C0E0C6E02C10BF041EC06F01A
:100E30001D0E0C6E03C10BF041EC06F01A0E57ECC0
:100E400006F0E8CF00F11B0E57EC06F0E8CF01F1F9
:100E50001C0E57EC06F0E8CF02F11D0E57EC06F021
:100E6000E8CF03F100C181F101C182F102C183F138
:100E700003C184F1240EAC6E900EAB6E240EAC6EEA
:100E8000080EB86E000EB06E1F0EAF6E0401806BC0
:100E9000816B0F01900EAB6E0F019D8A0301806B79
:100EA000816BA26B8B9207900001F28EF28C07B0DF
:100EB00074EF11F00EB055EF0CF003018051811961
:100EC0007F0BD8B474EF11F013EE00F081517F0B5B
:100ED000E126812BE7CFE8FFE00BD8B474EF11F0E7
:100EE00023EE82F0A2511F0BD926E7CFDFFFA22B02
:100EF000DF50780AD8A474EF11F007807DC100F1AB
:100F00007EC101F17FC102F180C103F10101040E34
:100F1000046F000E056F000E066F000E076FB0EC39
:100F200013F000AF9DEF07F00101030E7D6F000E7F
:100F30007E6F000E7F6F000E806F03018251720A78
:100F4000D8B455EF0CF08251520AD8B455EF0CF0DA
:100F50008251750AD8B455EF0CF08251630AD8B4A7
:100F600030EF0EF08251690AD8B437EF09F08251A0
:100F70007A0AD8B44AEF0AF08251490AD8B4D6EFB7
:100F800008F08251500AD8B4F4EF07F08251700A89
:100F9000D8B437EF08F08251540AD8B462EF08F0A1
:100FA0008251740AD8B4A8EF08F08251730AD8B4F9
:100FB00085EF0BF08251530AD8B4EAEF0BF065EFDE
:100FC0000EF0040114EE00F080517F0BE12682C484
:100FD000E7FF802B12000D0E826FE1EC07F00A0E86
:100FE000826FE1EC07F0120083C31EF184C31FF18E
:100FF00085C320F186C321F187C322F188C323F181
:1010000089C324F18AC325F18BC326F18CC327F150
:101010000101F5EC14F06CEC14F0160E0C6E00C12E
:101020000BF041EC06F0170E0C6E01C10BF041EC19
:1010300006F0180E0C6E02C10BF041EC06F0190E12
:101040000C6E03C10BF041EC06F000C179F101C157
:101050007AF102C17BF103C17CF100C17DF101C1D4
:101060007EF102C17FF103C180F1D6EF08F083C3A6
:101070001EF184C31FF185C320F186C321F187C30C
:1010800022F188C323F189C324F18AC325F18BC3DC
:1010900026F18CC327F10101F5EC14F06CEC14F08F
:1010A00000C179F101C17AF102C17BF103C17CF188
:1010B00000C17DF101C17EF102C17FF103C180F168
:1010C000D6EF08F083C31EF184C31FF185C320F15E
:1010D00086C321F187C322F188C323F189C324F198
:1010E0008AC325F18CC326F18DC327F10101F5ECEC
:1010F00014F06CEC14F00101000E046F000E056F8B
:10110000010E066F000E076FBFEC13F01A0E0C6E87
:1011100000C10BF041EC06F01B0E0C6E01C10BF090
:1011200041EC06F01C0E0C6E02C10BF041EC06F017
:101130001D0E0C6E03C10BF041EC06F000C181F1F5
:1011400001C182F102C183F103C184F1D6EF08F03D
:1011500083C31EF184C31FF185C320F186C321F12F
:1011600087C322F188C323F189C324F18AC325F1FF
:101170008CC326F18DC327F10101F5EC14F06CEC62
:1011800014F00101000E046F000E056F010E066FD2
:10119000000E076FBFEC13F000C181F101C182F1B5
:1011A00002C183F103C184F1D6EF08F0160E57ECAB
:1011B00006F0E8CF00F1170E57EC06F0E8CF01F18A
:1011C000180E57EC06F0E8CF02F1190E57EC06F0B6
:1011D000E8CF03F14AEC14F076EC12F00401730E40
:1011E000826FE1EC07F004012C0E826FE1EC07F056
:1011F00079C100F17AC101F17BC102F17CC103F137
:101200004AEC14F076EC12F00401730E826FE1ECFC
:1012100007F004012C0E826FE1EC07F01A0E57EC78
:1012200006F0E8CF00F11B0E57EC06F0E8CF01F115
:101230001C0E57EC06F0E8CF02F11D0E57EC06F03D
:10124000E8CF03F180EC0EF004012C0E826FE1EC8C
:1012500007F081C100F182C101F183C102F184C1B3
:1012600003F180EC0EF0EBEC07F065EF0EF00401FB
:10127000690E826FE1EC07F004012C0E826FE1EC45
:1012800007F00101040E006F000E016F000E026FE7
:10129000000E036F4AEC14F020C182F40401300EFA
:1012A0008227E1EC07F021C182F40401300E82278D
:1012B000E1EC07F022C182F40401300E8227E1EC58
:1012C00007F023C182F40401300E8227E1EC07F01D
:1012D00024C182F40401300E8227E1EC07F025C11D
:1012E00082F40401300E8227E1EC07F026C182F47B
:1012F0000401300E8227E1EC07F027C182F40401DB
:10130000300E8227E1EC07F004012C0E826FE1EC35
:1013100007F00101030E006F000E016F000E026F57
:10132000000E036F4AEC14F020C182F40401300E69
:101330008227E1EC07F021C182F40401300E8227FC
:10134000E1EC07F022C182F40401300E8227E1ECC7
:1013500007F023C182F40401300E8227E1EC07F08C
:1013600024C182F40401300E8227E1EC07F025C18C
:1013700082F40401300E8227E1EC07F026C182F4EA
:101380000401300E8227E1EC07F027C182F404014A
:10139000300E8227E1EC07F004012C0E826FE1ECA5
:1013A00007F00101160E006F000E016F000E026FB4
:1013B000000E036F4AEC14F020C182F40401300ED9
:1013C0008227E1EC07F021C182F40401300E82276C
:1013D000E1EC07F022C182F40401300E8227E1EC37
:1013E00007F023C182F40401300E8227E1EC07F0FC
:1013F00024C182F40401300E8227E1EC07F025C1FC
:1014000082F40401300E8227E1EC07F026C182F459
:101410000401300E8227E1EC07F027C182F40401B9
:10142000300E8227E1EC07F004012C0E826FE1EC14
:1014300007F0200EF86EF76AF66A04010900F5CF8E
:1014400082F4E1EC07F00900F5CF82F4E1EC07F05B
:101450000900F5CF82F4E1EC07F00900F5CF82F442
:10146000E1EC07F00900F5CF82F4E1EC07F00900A8
:10147000F5CF82F4E1EC07F00900F5CF82F4E1EC5E
:1014800007F00900F5CF82F4E1EC07F0EBEC07F090
:1014900065EF0EF08351630AD8A465EF0EF0845116
:1014A000610AD8A465EF0EF085516C0AD8A465EFE7
:1014B0000EF08651410A42E08651440A1BE08651F3
:1014C000420AD8B4B1EF0AF08651350AD8B4EFEF2A
:1014D0000FF08651360AD8B444EF10F08651370A1F
:1014E000D8B4ADEF10F08651380AD8B40BEF11F034
:1014F00065EF0EF00798079A04017A0E826FE1EC0F
:1015000007F00401780E826FE1EC07F00401640E2D
:10151000826FE1EC07F081A895EF0AF00401550E07
:10152000826FE1EC07F09AEF0AF004014C0E826F33
:10153000E1EC07F0EBEC07F065EF0EF00788079A97
:1015400004017A0E826FE1EC07F00401410E826F14
:10155000E1EC07F00401610E826FE1EC07F08BEF24
:101560000AF00798078A04017A0E826FE1EC07F00F
:101570000401420E826FE1EC07F00401610E826FFC
:10158000E1EC07F08BEF0AF001015967CFEF0AF0A9
:101590005A67CFEF0AF05B67CFEF0AF05C67E7EFBF
:1015A0000AF04267DBEF0AF04367DBEF0AF04467BB
:1015B000DBEF0AF04567E7EF0AF00101000E006F6C
:1015C000000E016F000E026F000E036F120001018A
:1015D000620E046F010E056F000E066F000E076F9E
:1015E00059C100F15AC101F15BC102F15CC103F1C3
:1015F000B0EC13F003BF44EF0BF00E0E57EC06F007
:10160000E8CF0CF10F0E57EC06F0E8CF0DF1100EFD
:1016100057EC06F0E8CF0EF1110E57EC06F0E8CFCC
:101620000FF1F9EC12F059C104F15AC105F15BC197
:1016300006F15CC107F1B0EC13F00782BDEC12F0CB
:10164000F9EC12F00792BDEC12F059C100F15AC149
:1016500001F15BC102F15CC103F10792BDEC12F034
:10166000CC0E046FE00E056F870E066F050E076F38
:10167000B0EC13F000C10CF101C10DF102C10EF18B
:1016800003C10FF17CEF0BF00101800E006F1A0E09
:10169000016F060E026F000E036F42C104F143C1D9
:1016A00005F144C106F145C107F1B0EC13F003AFF9
:1016B0005DEF0BF0A7EC14F012000E0E57EC06F0E5
:1016C000E8CF0CF10F0E57EC06F0E8CF0DF1100E3D
:1016D00057EC06F0E8CF0EF1110E57EC06F0E8CF0C
:1016E0000FF142C100F143C101F144C102F145C112
:1016F00003F10782BDEC12F00CC100F10DC101F144
:101700000EC102F10FC103F112000401730E826FCA
:10171000E1EC07F004012C0E826FE1EC07F0078486
:1017200055C159F156C15AF157C15BF158C15CF12D
:101730003EC142F13FC143F140C144F141C145F1D5
:101740004AC14CF14BC14DF10794ABEC0BF0EBEC03
:1017500007F065EF0EF059C100F15AC101F15BC10C
:1017600002F15CC103F101014AEC14F076EC12F0D5
:101770000401630E826FE1EC07F004012C0E826F0E
:10178000E1EC07F042C100F143C101F144C102F1B3
:1017900045C103F101014AEC14F076EC12F00401AA
:1017A000660E826FE1EC07F004012C0E826FE1EC13
:1017B00007F0A7EC14F04CC100F14DC101F101019B
:1017C0004AEC14F076EC12F00401740E826FE1EC36
:1017D00007F012000F820401530E826FE1EC07F054
:1017E00004012C0E826FE1EC07F083C31EF184C369
:1017F0001FF185C320F186C321F187C322F188C37D
:1018000023F189C324F18AC325F18BC326F18CC34C
:1018100027F10101F5EC14F06CEC14F000C159F162
:1018200001C15AF102C15BF103C15CF18EC31EF12B
:101830008FC31FF190C320F191C321F192C322F114
:1018400093C323F194C324F195C325F196C326F1E4
:1018500097C327F10101F5EC14F06CEC14F000C112
:1018600042F101C143F102C144F103C145F1E8EC89
:1018700014F099C323F19AC324F19BC325F19CC3AF
:1018800026F19DC327F10101F5EC14F06CEC14F086
:1018900000C14CF101C14DF1ABEC0BF004012C0E79
:1018A000826FE1EC07F05CEF0CF08251520A03E129
:1018B0000E825CEF0CF00E928251750A03E10F84E8
:1018C00063EF0CF00F948251550A03E10F866AEF23
:1018D0000CF00F9607840FB2C7EF0CF00FA4B3EF14
:1018E0000CF0A5C159F1A6C15AF1A7C15BF1A8C17D
:1018F0005CF1A9C15DF1AAC15EF1ABC15FF1ACC100
:1019000060F1ADC161F1AEC162F1AFC163F1B0C1CF
:1019100064F1B1C165F1B2C166F1B3C167F1B4C19F
:1019200068F1B5C169F1B6C16AF1B7C16BF1B8C16F
:101930006CF1B9C16DF1BAC16EF1BBC16FF1BCC13F
:1019400070F1BDC171F1BEC172F1BFC173F1C0C10F
:1019500074F1C1C175F1C2C176F1C3C177F1C4C1DF
:1019600078F1BBEF0CF055C159F156C15AF157C18E
:101970005BF158C15CF13EC142F13FC143F140C14E
:1019800044F141C145F14AC14CF14BC14DF10794BD
:101990000EA0E9EF0CF001018167D6EF0CF0826731
:1019A000D6EF0CF08367D6EF0CF08467DAEF0CF01B
:1019B000E9EF0CF0C4EC0AF081C104F182C105F139
:1019C00083C106F184C107F1B0EC13F003BF2DEF22
:1019D0000EF0C4EC0AF00101000E046F000E056F5A
:1019E000010E066F000E076FDEEC13F00FA400EF80
:1019F0000DF00401750E826FE1EC07F005EF0DF0BC
:101A00000401720E826FE1EC07F004012C0E826F6C
:101A1000E1EC07F04AEC14F01D6714EF0DF004013F
:101A2000200E826F17EF0DF004012D0E826FE1EC96
:101A300007F024C182F40401300E8227E1EC07F0A4
:101A400025C182F40401300E8227E1EC07F0040185
:101A50002E0E826FE1EC07F026C182F40401300EF5
:101A60008227E1EC07F027C182F40401300E8227BF
:101A7000E1EC07F004016D0E826FE1EC07F0040168
:101A80002C0E826FE1EC07F042C100F143C101F17D
:101A900044C102F145C103F101014AEC14F076ECB6
:101AA00012F00401480E826FE1EC07F004017A0E97
:101AB000826FE1EC07F004012C0E826FE1EC07F07D
:101AC00059C100F15AC101F15BC102F15CC103F1DE
:101AD00001014AEC14F076EC12F00401630E826FFF
:101AE000E1EC07F004012C0E826FE1EC07F059C124
:101AF00000F15AC101F15BC102F15CC103F10101C6
:101B00000A0E046F000E056F000E066F000E076FC1
:101B1000BFEC13F0000E046F120E056F000E066F7F
:101B2000000E076FDEEC13F04AEC14F01EC182F4D5
:101B30000401300E8227E1EC07F01FC182F404019A
:101B4000300E8227E1EC07F020C182F40401300E50
:101B50008227E1EC07F021C182F40401300E8227D4
:101B6000E1EC07F022C182F40401300E8227E1EC9F
:101B700007F023C182F40401300E8227E1EC07F064
:101B800024C182F40401300E8227E1EC07F0040145
:101B90002E0E826FE1EC07F025C182F40401300EB5
:101BA0008227E1EC07F026C182F40401300E82277F
:101BB000E1EC07F027C182F40401300E8227E1EC4A
:101BC00007F00401730E826FE1EC07F004012C0EA4
:101BD000826FE1EC07F0A7EC14F04CC100F14DC1AD
:101BE00001F18FEC0FF00EB2F9EF0DF00EA02BEF1C
:101BF0000EF004012C0E826FE1EC07F0200EF86E5F
:101C0000F76AF66A04010900F5CF82F4E1EC07F007
:101C10000900F5CF82F4E1EC07F00900F5CF82F47A
:101C2000E1EC07F00900F5CF82F4E1EC07F00900E0
:101C3000F5CF82F4E1EC07F00900F5CF82F4E1EC96
:101C400007F00900F5CF82F4E1EC07F00900F5CFC9
:101C500082F4E1EC07F0EBEC07F00E9065EF0EF08C
:101C60000401630E826FE1EC07F004012C0E826F19
:101C7000E1EC07F06BEC0EF004012C0E826FE1EC4E
:101C800007F0DEEC0EF004012C0E826FE1EC07F0A1
:101C90005AEC0FF004012C0E826FE1EC07F0010109
:101CA000F80E006FCD0E016F660E026F030E036F0C
:101CB00080EC0EF004012C0E826FE1EC07F070EC6A
:101CC0000FF0EBEC07F065EF0EF00301A26B07904D
:101CD0000F9274EF11F0D8900E0E57EC06F0E8CF8B
:101CE00000F10F0E57EC06F0E8CF01F1100E57ECA3
:101CF00006F0E8CF02F1110E57EC06F0E8CF03F141
:101D00000101000E046F000E056F010E066F000E3C
:101D1000076FDEEC13F04AEC14F01EC182F40401EC
:101D2000300E8227E1EC07F01FC182F40401300E6F
:101D30008227E1EC07F020C182F40401300E8227F3
:101D4000E1EC07F021C182F40401300E8227E1ECBE
:101D500007F022C182F40401300E8227E1EC07F083
:101D600023C182F40401300E8227E1EC07F024C184
:101D700082F40401300E8227E1EC07F025C182F4E1
:101D80000401300E8227E1EC07F004012E0E826F71
:101D9000E1EC07F026C182F40401300E8227E1EC69
:101DA00007F027C182F40401300E8227E1EC07F02E
:101DB00004016D0E826FE1EC07F01200120E57EC79
:101DC00006F0E8CF00F1130E57EC06F0E8CF01F172
:101DD000140E57EC06F0E8CF02F1150E57EC06F0A2
:101DE000E8CF03F101010A0E046F000E056F000E2B
:101DF000066F000E076FBFEC13F0000E046F120E9B
:101E0000056F000E066F000E076FDEEC13F04AEC54
:101E100014F01EC182F40401300E8227E1EC07F0B9
:101E20001FC182F40401300E8227E1EC07F020C1CB
:101E300082F40401300E8227E1EC07F021C182F424
:101E40000401300E8227E1EC07F022C182F4040184
:101E5000300E8227E1EC07F023C182F40401300E3A
:101E60008227E1EC07F024C182F40401300E8227BE
:101E7000E1EC07F004012E0E826FE1EC07F025C1C2
:101E800082F40401300E8227E1EC07F026C182F4CF
:101E90000401300E8227E1EC07F027C182F404012F
:101EA000300E8227E1EC07F00401730E826FE1EC43
:101EB00007F012000A0E57EC06F0E8CF00F10B0E07
:101EC00057EC06F0E8CF01F10C0E57EC06F0E8CF26
:101ED00002F10D0E57EC06F0E8CF03F18FEF0FF093
:101EE000060E57EC06F0E8CF00F1070E57EC06F0AF
:101EF000E8CF01F1080E57EC06F0E8CF02F1090E29
:101F000057EC06F0E8CF03F18FEF0FF00101A7ECDB
:101F100014F007844AC100F14BC101F1079401019B
:101F2000E80E046F800E056F000E066F000E076F3F
:101F3000BFEC13F0000E046F040E056F000E066F69
:101F4000000E076FDEEC13F0880E046F130E056FA2
:101F5000000E066F000E076FB0EC13F00A0E046F50
:101F6000000E056F000E066F000E076FDEEC13F01B
:101F70004AEC14F001011D67C3EF0FF00401200EBD
:101F8000826FC6EF0FF004012D0E826FE1EC07F0B7
:101F900024C182F40401300E8227E1EC07F025C150
:101FA00082F40401300E8227E1EC07F026C182F4AE
:101FB0000401300E8227E1EC07F004012E0E826F3F
:101FC000E1EC07F027C182F40401300E8227E1EC36
:101FD00007F00401430E826FE1EC07F0120087C3A3
:101FE0001EF188C31FF189C320F18AC321F18BC37D
:101FF00022F18CC323F18DC324F18EC325F190C34C
:1020000026F191C327F101011D6BF5EC14F06CEC86
:1020100014F00101000E046F000E056F010E066F33
:10202000000E076FBFEC13F00E0E0C6E00C10BF02C
:1020300041EC06F00F0E0C6E01C10BF041EC06F006
:10204000100E0C6E02C10BF041EC06F0110E0C6E7E
:1020500003C10BF041EC06F004017A0E826FE1EC53
:1020600007F004012C0E826FE1EC07F00401350E3D
:10207000826FE1EC07F004012C0E826FE1EC07F0B7
:102080006BEC0EF09AEF0AF087C31EF188C31FF1C4
:1020900089C320F18AC321F18BC322F18CC323F1C0
:1020A0008DC324F18EC325F190C326F191C327F18E
:1020B00001011D6BF5EC14F06CEC14F0880E046F4C
:1020C000130E056F000E066F000E076FB4EC13F0D1
:1020D000000E046F040E056F000E066F000E076FF2
:1020E000BFEC13F00101E80E046F800E056F000EC7
:1020F000066F000E076FDEEC13F00A0E0C6E00C1C7
:102100000BF041EC06F00B0E0C6E01C10BF041EC34
:1021100006F00C0E0C6E02C10BF041EC06F00D0E39
:102120000C6E03C10BF041EC06F004017A0E826FD5
:10213000E1EC07F004012C0E826FE1EC07F00401E2
:10214000360E826FE1EC07F004012C0E826FE1EC99
:1021500007F05AEC0FF09AEF0AF087C31EF188C31C
:102160001FF189C320F18AC321F18BC322F18CC3F3
:1021700023F18DC324F18FC325F190C326F191C3C0
:1021800027F10101F5EC14F06CEC14F0000E046F73
:10219000120E056F000E066F000E076FBFEC13F0F6
:1021A00001010A0E046F000E056F000E066F000E8F
:1021B000076FDEEC13F0120E0C6E00C10BF041EC59
:1021C00006F0130E0C6E01C10BF041EC06F0140E7C
:1021D0000C6E02C10BF041EC06F0150E0C6E03C143
:1021E0000BF041EC06F004017A0E826FE1EC07F08F
:1021F00004012C0E826FE1EC07F00401370E826FB0
:10220000E1EC07F004012C0E826FE1EC07F0DEEC4C
:102210000EF09AEF0AF087C31EF188C31FF189C33D
:1022200020F18AC321F18BC322F18CC323F18DC32A
:1022300024F18EC325F190C326F191C327F101014A
:102240001D6BF5EC14F06CEC14F0880E046F130E9B
:10225000056F000E066F000E076FB4EC13F0000E52
:10226000046F040E056F000E066F000E076FBFECC3
:1022700013F00101E80E046F800E056F000E066F6B
:10228000000E076FDEEC13F0060E0C6E00C10BF0B3
:1022900041EC06F0070E0C6E01C10BF041EC06F0AC
:1022A000080E0C6E02C10BF041EC06F0090E0C6E2C
:1022B00003C10BF041EC06F004017A0E826FE1ECF1
:1022C00007F004012C0E826FE1EC07F00401380ED8
:1022D000826FE1EC07F004012C0E826FE1EC07F055
:1022E00070EC0FF09AEF0AF081A832EF12F007A815
:1022F000EBEF11F00101800E006F1A0E016F060E58
:10230000026F000E036F3EC104F13FC105F140C1F1
:1023100006F141C107F1B0EC13F003BF32EF12F048
:1023200070EC12F03EC100F13FC101F140C102F179
:1023300041C103F10782BDEC12F00CC104F10DC1E3
:1023400005F10EC106F10FC107F1F80E006FCD0EB9
:10235000016F660E026F030E036FB0EC13F00E0EEA
:102360000C6E00C10BF041EC06F00F0E0C6E01C1BB
:102370000BF041EC06F0100E0C6E02C10BF041ECBC
:1023800006F0110E0C6E03C10BF041EC06F0078451
:102390000101A7EC14F04AC100F14BC101F107940F
:1023A0000A0E0C6E00C10BF041EC06F00B0E0C6E29
:1023B00001C10BF041EC06F00C0E0C6E02C10BF0EB
:1023C00041EC06F00D0E0C6E03C10BF041EC06F073
:1023D000079832EF12F007AA32EF12F007840101DA
:1023E000A7EC14F04AC100F14BC101F10794060EAD
:1023F0000C6E00C10BF041EC06F0070E0C6E01C133
:102400000BF041EC06F0080E0C6E02C10BF041EC33
:1024100006F0090E0C6E03C10BF041EC06F00784C8
:1024200055C100F156C101F157C102F158C103F184
:102430000794120E0C6E00C10BF041EC06F0130E67
:102440000C6E01C10BF041EC06F0140E0C6E02C1D3
:102450000BF041EC06F0150E0C6E03C10BF041ECD5
:1024600006F0079A0401805181197F0B0BE09EA8AA
:1024700009D014EE00F081517F0BE126E750812B4B
:102480000F01AD6E57EF07F00CC100F10DC101F166
:102490000EC102F10FC103F1000E046F000E056FB3
:1024A000010E066F000E076FDEEC13F01DA16FEF3B
:1024B00012F01451D8B46FEF12F00CC100F10DC13D
:1024C00001F10EC102F10FC103F1000E046F000E05
:1024D000056F0A0E066F000E076FDEEC13F0120098
:1024E00001010C6B0D6B0E6B0F6B12001EC182F4A1
:1024F0000401300E8227E1EC07F01FC182F40401D1
:10250000300E8227E1EC07F020C182F40401300E86
:102510008227E1EC07F021C182F40401300E82270A
:10252000E1EC07F022C182F40401300E8227E1ECD5
:1025300007F023C182F40401300E8227E1EC07F09A
:1025400024C182F40401300E8227E1EC07F025C19A
:1025500082F40401300E8227E1EC07F026C182F4F8
:102560000401300E8227E1EC07F027C182F4040158
:10257000300E8227E1EC07F012000101005305E163
:10258000015303E1025301E1002B80EC13F0A7ECAF
:1025900014F02C51006F2D51016F420E046F4B0E41
:1025A000056F000E066F000E076FBFEC13F000C141
:1025B00004F101C105F102C106F103C107F10CC12B
:1025C00000F10DC101F10EC102F10FC103F107B21B
:1025D000EEEF12F0B4EC13F0F0EF12F0B0EC13F0F9
:1025E00000C10CF101C10DF102C10EF103C10FF1E7
:1025F0001200A7EC14F04CC100F14DC101F1060E20
:1026000057EC06F0E8CF04F1070E57EC06F0E8CFE0
:1026100005F1080E57EC06F0E8CF06F1090E57EC6D
:1026200006F0E8CF07F1B0EC13F000C118F101C1DA
:1026300019F102C11AF103C11BF1290E046F000E3A
:10264000056F000E066F000E076FBFEC13F0EE0E65
:10265000046F430E056F000E066F000E076FB4EC9B
:1026600013F018C104F119C105F11AC106F11BC11B
:1026700007F1BFEC13F000C110F101C111F102C16B
:1026800012F103C113F1120E57EC06F0E8CF04F17A
:10269000130E57EC06F0E8CF05F1140E57EC06F0D8
:1026A000E8CF06F1150E57EC06F0E8CF07F10D0E56
:1026B000006F000E016F000E026F000E036FBFEC83
:1026C00013F0180E046F000E056F000E066F000E5B
:1026D000076FDEEC13F010C104F111C105F112C156
:1026E00006F113C107F1B4EC13F06A0E046F2A0E61
:1026F000056F000E066F000E076FB0EC13F01200AE
:10270000BF0EFA6E200E2D6F2C6BD890003701375C
:1027100002370337D8B091EF13F02D2F86EF13F067
:102720002C072D070353D8B412000331070B80097F
:10273000326F03390F0B010F2C6F80EC5FF0336F9A
:102740002C0580EC5FF0335D335F2C6B3233D8B0F7
:102750002C272C3332A9A6EF13F033512C2712006B
:10276000CCEC14F0D8B0120003510719286F8FEC8D
:1027700014F0D8900751031928AF800F1200286B6E
:10278000B3EC14F0D8A0C9EC14F0D8B012009EEC51
:1027900014F0A7EC14F01F0E296FDFEC14F00B35CA
:1027A000D8B08FEC14F0D8A00335D8B01200292F80
:1027B000CDEF13F028B1B6EC14F01200286B0451E1
:1027C0000511061107110008D8A0B3EC14F0D8A029
:1027D000C9EC14F0D8B01200086B096B0A6B0B6BD4
:1027E000DFEC14F01F0E296FDFEC14F007510B5DC6
:1027F000D8A407EF14F006510A5DD8A407EF14F02F
:102800000551095DD8A407EF14F00451085DD8A064
:102810001AEF14F00451085F0551D8A0053D095F77
:102820000651D8A0063D0A5F0751D8A0073D0B5FAF
:10283000D8900081292FF4EF13F028B1B6EC14F0F2
:10284000286BB3EC14F0D890E3EC14F007510B5D57
:10285000D8A437EF14F006510A5DD8A437EF14F06E
:102860000551095DD8A437EF14F00451085DD8A0D4
:1028700046EF14F0003F46EF14F0013F46EF14F02E
:10288000023F46EF14F0032BD8B4120028B1B6EC87
:1028900014F012000101286BB3EC14F0D8B0120050
:1028A000E8EC14F0200E296F0037013702370337A8
:1028B00011EE27F00A0E2A6FE7360A0EE75CD8B051
:1028C000E76EE5522A2F5CEF14F0292F54EF14F035
:1028D00028B11D81D890120001010A0E286F200E28
:1028E000296F11EE1DF028512A6F0A0ED890E6527A
:1028F000D8B0E726E7322A2F77EF14F003330233FC
:1029000001330033292F71EF14F0E750FF0FD8A0E7
:102910000335D8B012001DB1B6EC14F0120004510A
:1029200000270551D8B0053D01270651D8B0063D16
:1029300002270751D8B0073D032712000051086F46
:102940000151096F02510A6F03510B6F120001010F
:10295000006B016B026B036B12000101046B056BD2
:10296000066B076B12000335D8A012000351800BD1
:10297000001F011F021F031F003FC6EF14F0013F9D
:10298000C6EF14F0023FC6EF14F0032B282B0325EB
:1029900012000735D8A012000751800B041F051F35
:1029A000061F071F043FDCEF14F0053FDCEF14F0B7
:1029B000063FDCEF14F0072B282B07251200003709
:1029C000013702370337083709370A370B37120048
:1029D00001011D6B1E6B1F6B206B216B226B236B28
:1029E000246B256B266B276B12001E510F0B1E6F7D
:1029F0001F510F0B1F6F20510F0B206F21510F0B19
:102A0000216F22510F0B226F23510F0B236F245183
:102A10000F0B246F25510F0B256F26510F0B266FBF
:082A200027510F0B276F120074
:10BF0000E844F926000C160C2B0C3F0C520C640C68
:10BF1000760C860C960CA50CB30CC10CCF0CDC0C6B
:06BF2000E80CF40C000C1B
:00000001FF
